:0400000002008F3239
:01000B0032C2
:0100130032BA
:01001B0032B2
:0100230032AA
:100080004D50332D4C434420563A312E31300075BB
:1000900081201200A61201C89000801201F1748024
:1000A0001201380200ECC2B0D2B122D2B1D2B0E516
:1000B000B05403B403F9E5B05403B4030280F7B4B9
:1000C00001ED20B0FDC2B022D2B1C0F075F008D26F
:1000D000B030B0FDA2B1400320B10D20B0F8C2B0E5
:1000E00033D5F0EBD0F0C322D3D0F02211AB11C83E
:1000F00040FAB420F7C2B1D2B030B0FD20B0FDC29A
:10010000B011C840E7B40107748012013880E6B42A
:10011000020774C012013880DCB4030512024D805E
:10012000D4B4040512025B80CCB40507740112013B
:100130003880C212014B80BD12016AC2B5C2B4F54B
:100140009000D2B700C2B71201AD2212016AD2B537
:10015000C2B4C083C0829002B893D082D083F5909D
:1001600000D2B700C2B71201BA22C0E0C0F075F0E9
:10017000FF15F0E5F060171201BAC2B5D2B400D293
:10018000B7001201BAE590C2B720E7E5C2B4D0F0DB
:10019000D0E022C0E0740A1201BA1470FAD0E02252
:1001A000C0E074C81201BA1470FAD0E022C0E07442
:1001B000321201BA1470FAD0E022C0E0740A14704E
:1001C000FDD0E022380C0106C2B7C2B5C2B431A0DE
:1001D0009001C4740093313831AD313831BA75F0C3
:1001E000047400933138A315F0E5F070F41202693D
:1001F000227400936009314BA315F0E5F080F222E0
:10020000540F2430C0E0C3943A4006D0E02407C025
:10021000E0D0E0314B22C0E0C45100D0E0C0E0515A
:1002200000D0E0222020202020202020202020207C
:1002300020202020202020202020202020202020BE
:100240002020202020202020202020200074803109
:100250003890022431F1748031382274C0313890E2
:10026000022431F174C03138229002887440313850
:10027000740675F008C3A47800F9E893314B0819A7
:10028000E970F77480313822110E11111F1111001D
:10029000110E111111110E000A11111111110E0080
:1002A00010181C1E1C1810001B1B1B1B1B1B1B00EB
:1002B0000000040E1F001F002001020304050607B2
:1002C00008090A0B0C0D0E0F101112131415161736
:1002D00018191A1B1C1D1E1F202122232425262726
:1002E00028292A2B2C2D2E2F303132333435363716
:1002F00038393A3B3C3D3E3F404142434445464706
:1003000048494A4B4C4D4E4F5051525354555657F5
:1003100058595A5B2F5D5E5F606162636465666712
:1003200068696A6B6C6D6E6F7071727374757677D5
:1003300078797A7B7C7DEDFFFFFFFFFFFFFFFFFFFA
:10034000FFFFFFFFFFFFFFFFFF2727FFFFFFFFFF6D
:10035000FFFFFFFFFFFFFFFF2021ECDBDB5C7CDB0F
:100360002263617FDB2D72B0DFDB323327E4DBA554
:100370002C31DF7EDBDBDB3F414141410041DB4390
:100380004545454549494949444E4F4F4F4F0178EE
:10039000305555550259DBE261616161E161DB6312
:1003A00065656565696969696F6E6F6F6F6FEFFD90
:0803B00030757575F579DB79F4
:00000001FF
